:020000040000FA
:100000005634120012907800FFFFFF00FFFFFF0040
:10001000FFFFFF00FFFFFF00FFFFFF00FFFFFF00EC
:10002000FFFFFF00FFFFFF00FFFFFF00FFFFFF00DC
:10003000FFFFFF00FFFFFF00FFFFFF00FFFFFF00CC
:10004000FFFFFF00FFFFFF00FFFFFF00FFFFFF00BC
:103FF000FFFFFF00FFFFFF0054769800981032008B
:0200000400FFFB
:10F800003412000078560000FFFF0000FFFF0000E8
:10F81000FFFF0000FFFF0000FFFF0000FFFF0000F0
:10F82000FFFF0000FFFF0000FFFF0000FFFF0000E0
:10F83000FFFF0000FFFF0000FFFF0000FFFF0000D0
:10F84000FFFF0000FFFF0000FFFF0000FFFF0000C0
:10FFF000FFFF0000FFFF00008709000043650000CD
:0200000401F009
:100000000FC100003F000000A38300000F3100007B
:0C0010000F3300000500000003C00000DA
:00000001FF
